:040000000FC0FECF60
:10000400FDCFFCCFFBCF3CC0F9CFF8CFF7CFF6CF75
:10001400F5CFF4CFF3CFF2CFF1CF0000F894EE2771
:10002400ECBBE5BFF8E1A895A4B7A77FA4BFF1BDD9
:10003400E1BD8DE0A2E0ED938A95E9F780E8A0E6C2
:10004400ED938A95E9F7EEE1F0E0859195910097BB
:1000540061F0A591B59105901590BF01F00105904F
:100064000D920197E1F7FB01F0CFE0E0E1BBE0E0A6
:10007400E2BBE0E0E3BBEFEDEDBFC0E8D0E070C071
:10008400EA93FA93EFB7EA93E0E0E2BFF101319625
:100094001F01E1E0E61541F4E4E6F0E0E215F305C2
:1000A40010F4C398662406C0E4E1F0E0E215F30519
:1000B40009F4C3984214530430F4E1E0E71519F449
:1000C400E0E0E61509F001C032D1E991EFBFF99102
:1000D400E9911895E881E066E7B980E28A95F1F73D
:1000E400369A349BFECF349AE5B1219608956AD1AD
:1000F40010E01233B8F480E68A95F1F7E1E0EA9370
:10010400E9DF0E2F80E68A95F1F7A895E02FEE7FC0
:10011400EF9311D1DFDFEE7FAF91EA1709F010E022
:100124001F5FE7CFE02F51D10895A895E199FECF45
:10013400E0E0ECBBE981EEBBE881EDBBF894E29A28
:10014400E19AE199FECF789422960895A895E199D1
:10015400FECFE881EEBBE1E0ECBBEDB32196089560
:1001640000E010E020E030E0E0E8E6BDE0E0E6BDDD
:10017400E8BBE7BBEABDE5E0E3BFE0E0E2BFE9BD21
:10018400E8BDE7BDE0BFECBDEFBDEEBDEBBDEDBD31
:10019400EBBFE5BFE2E0E9BFE0E0EDB9E0E8E8B9D4
:1001A400E0E0E3B9E9E3E1BDE9E2E1BDE4B3E37032
:1001B400E4BBA29AE0E6E7B9E4E8E6B9E3B1EF7597
:1001C400E3B9C498BC9AC398BB9A7894A895B19B98
:1001D40046C010E0ACD0A895C39B03C0A895AED090
:1001E400FBCF85DFE23318F4A895A8D0FACFABD0C3
:1001F40050F0A895A3D0AAD00F3F10F4101708F020
:1002040001C0102FF4CFE0E0EA931A938EDF8FD071
:10021400C39B03C093D0A895FBCF69DFE23318F4E6
:10022400A8958CD0FACF92D0033320F0E12FE2537B
:10023400E01708F003C07FD0EFEF02C07CD0E0E00D
:10024400EA9373DF80D020F0A89578D07FD0FACFDE
:100254006ED0C39B03C072D0A895FBCFA895E0E0F5
:10026400EA9374DF1E2F1F3F09F410E064D06EDFA1
:100274003E2FE0E4F0E06DD018F4A8955FD0F9CFFC
:10028400C49AA895772059F55ED040F122243324EE
:100294005AD010F061D008F003C0A8954FD0F8CF21
:1002A40026DFE23310F458D008F003C0A89546D0F6
:1002B400F7CF49D010F050D008F010C047D0101735
:1002C40010F40F3F08F005C0E0E0EA930A932DDF35
:1002D400102F303009F4C498E1E07E2E25C0303070
:1002E40041F4B19B06C0A89529D021D0E1E06E2E3F
:1002F400F8CF2CD0023320F4772420E0C49A14C021
:10030400E02FF0E0A12FB0E0AE1BBF0BE8E0F0E07F
:1003140046D0E259FF4F2F01A02FA5502A1718F4F9
:10032400E0EDF7E01F01202F09D0ABCFFFCF22244F
:100334003324C39A0895E1E0EA930895EAE0F0E0F3
:10034400FA93EA930CC0D3DEE3330895D0DE0E2F84
:1003540008952E163F060895E0E2F0E0FACFE99101
:10036400F991309639F080E699E00197F1F7A89574
:100374003197C9F70895F195E195F04008950A2E53
:100384001B2E81E1AA27BB1B05C010F4A00DB11DD3
:10039400B695A795F795E7958A95B9F7089504D08A
:1003A400EEDF0EF4E8DF0895E894F7FF02C0E3DF20
:1003B4006894B7FF06C0A095B095119600F8039411
:1003C40000FA08951A930A930895099119910895CA
:00000001FF
